:020000040000FA
:040000008A01052844
:08000800152A0730831298133A
:10001000831607309C009D019B01850186010730F6
:1000200081008312850186013D3081001430A300D8
:100030008B178B16A601A701A801A901AA01AB0184
:10004000A20100222608382022083220860004223D
:100050000822082208220822A20A2208053C031DC1
:100060002428202882075F286128632865286728BC
:100070008207692874287F288A289528A028AB2819
:10008000B628C128CC28D728E228ED28F82803294B
:100090000E29192924292F293A29452950295B2974
:1000A000662971297C29872992299D29A829B329A4
:1000B000BE29C929D429DF29EA29F5291A282708C0
:1000C000080028080800290808002A0808002B084A
:1000D00008007C30A7008230A8008230A90082305E
:1000E000AA007C30AB0008000030A7008430A800D4
:1000F000FE30A9008030AA000030AB000800843038
:10010000A700C230A800A230A9009230AA008C300B
:10011000AB0008004430A7008230A8009230A9004C
:100120009230AA006C30AB0008001030A7001830E5
:10013000A8001430A900FE30AA001030AB0008005F
:100140005E30A7009230A8009230A9009230AA0039
:100150006230AB0008007C30A7009230A8009230DB
:10016000A9009230AA006430AB0008008230A700DA
:100170004230A8002230A9001230AA000E30AB0095
:1001800008006C30A7009230A8009230A90092308D
:10019000AA006C30AB0008004C30A7009230A800D9
:1001A0009230A9009230AA007C30AB000800FC30ED
:1001B000A7001230A8001230A9001230AA00FC30AB
:1001C000AB000800FE30A7009230A8009230A900D2
:1001D0009230AA006C30AB0008007C30A70082305F
:1001E000A8008230A9008230AA004430AB00080089
:1001F000FE30A7008230A8008230A9008230AA0019
:100200007C30AB000800FE30A7009230A80092308E
:10021000A9009230AA008230AB000800FE30A7008F
:100220001230A8001230A9001230AA000230AB0030
:1002300008007C30A7009230A8009230A9009230CC
:10024000AA007430AB000800FE30A7001030A800F0
:100250001030A9001030AA00FE30AB0008000030BA
:10026000A7008230A800FE30A9008230AA0000302A
:10027000AB0008007030A7008030A8008030A900D3
:100280008030AA007E30AB000800FE30A70010309E
:10029000A8002830A9004430AA008230AB00080032
:1002A000FE30A7008030A8008030A9008030AA006E
:1002B0008030AB000800FE30A7000430A8001830E2
:1002C000A9000430AA00FE30AB000800FE30A700F1
:1002D0000830A8001030A9002030AA00FE30AB0082
:1002E0000800FA30A7001230A8002230A9004230DE
:1002F000AA00FA30AB0008007C30A7008230A800CA
:100300008230A9008230AA007C30AB000800FE30A9
:10031000A7001230A8001230A9001230AA000C3039
:10032000AB0008007C30A7008230A800A230A900F2
:100330004230AA00BC30AB000800FE30A7001230EB
:10034000A8003230A9005230AA008C30AB0008005F
:100350004C30A7009230A8009230A9009230AA0039
:100360006430AB0008000230A7000230A800FE3065
:10037000A9000230AA000230AB0008007E30A700BE
:100380008030A8008030A9008030AA007E30AB0009
:1003900008003E30A7004030A8008030A90040305F
:1003A000AA003F30AB000800FE30A7004030A80094
:1003B0003030A9004030AA00FE30AB000800C63043
:1003C000A7002830A8001030A9002830AA00C630A5
:1003D000AB0008000630A7000830A800F030A900E4
:1003E0000830AA000630AB000800C230A700A230D7
:1003F000A8009230A9008A30AA008630AB0008001D
:10040000851410228510080005151022051108001A
:100410000F30A000A100A10B0B2AA00B0A2A080094
:10042000FA30A100A10B122A0800A400030EA500B7
:100430003D308100A30B1F2AA60A1430A300250E0D
:0A0440008300A40E240E0B11090026
:00000001FF
